:100000000C94D6010C94F1010C9492040C946E049F
:100010000C94F1010C9427110C94F1010C94F10152
:100020000C94F1010C94F1010C946A110C94F101FF
:100030000C94F1010C94F1010C94F1010C94F10178
:100040000C94F1010C94F1010C94F1010C94F10168
:100050000C94F1010C94F1010C9431051D5A3440BB
:10006000E17A34406ABC344091ED34407D3F354004
:10007000A47035402DB23540F2D23540B6F335404C
:100080003F353640666636408D97364017D9364044
:10009000643B3740EE7C374014AE37409EEF37402C
:1000A000B0723840E926394021B03A4093183C40BC
:1000B000350060008000B0001D013D015A017A0149
:1000C0009701B901DA01F901160240026D028202BC
:1000D000A202EF023203B003F203AA03A703A403B0
:1000E000A1039E039B039803940391038D038A034A
:1000F000860382037E037B03770372036E036A0326
:10010000660361035D03580353034F034A0345032A
:1001100040033B03360330032B03260320031B035A
:1001200015030F030A030403FE02F802F202EC02B5
:10013000E602DF02D902D302CC02C602BF02B90234
:10014000B202AC02A5029E02970291028A028302C9
:100150007C0275026E02680261025A0253024C026E
:1001600045023E0237023002290222021B0215021A
:100170000E0207020002F901F201EC01E501DE01C5
:10018000D801D101CB01C401BE01B701B101AA015F
:10019000A4019E01980192018C01860180017A01DF
:1001A00074016E01680163015D01580152014D0146
:1001B000470142013D01380133012E01290124018B
:1001C0001F011A01150111010C0108010301FF00B3
:1001D000FB00F600F200EE00EA00E600E200DE00BE
:1001E000DB00D700D300CF00CC00C800C500C200A0
:1001F000BE00BB002F03390342034B0353035C03D0
:1002000064036C0373037B03820388038F039503EA
:100210009B0326031C0312030703FD02F202E702FD
:10022000DC02D002C502B902AD02A1029502890228
:100230007C027002630257024A023E023202250229
:1002400019020C020002F401E801DC01D001C40132
:10025000B801AD01A20196018C01810176016C010A
:10026000620158014E0144013B0132012901200184
:1002700017010F010701FF00F700F000E900E1009E
:10028000DB00D400CD00C700C100BB00510A802AAA
:100290000000000A510A000059551801111E111BD7
:1002A000500B411B411F1101511F511B0000000049
:1002B00000000000000000000000510F91394114BF
:1002C0009131411E410E411D500F8020101548866E
:1002D0004014780570855115510E5195518E21901D
:1002E00081205015484450C528C0282009500000DE
:1002F000000000000000000054494D4552004155E7
:10030000544F004D414E00534554004F5054494FF7
:100310004E004D53544F50004D53544152540041E0
:1003200053544152540053484F4F5400574149547D
:1003300000434F554E540042555A5A4552004F4EB5
:10034000004F464600434C49434B004F4E004F463A
:1003500046004C4544004F4646004F4E004C49472E
:100360004854004155544F0054454D50000001027F
:1003700003040504050001020304050203000159FA
:10038000594D4D4444004D4D444459590044444D49
:100390004D5959003234480031324800313248005A
:1003A00032344800323448003132480011241FBE34
:1003B000CFEFD4E0DEBFCDBF11E0A0E0B1E0E8EBCD
:1003C000F6E202C005900D92AE33B107D9F711E005
:1003D000AEE3B1E001C01D92AC3AB107E1F70C9475
:1003E0002D070C94000040E050E08B9A839A809196
:1003F0007A00806880937A0080917A00806480938C
:100400007A0080917A0084FFFCCF30E080917A00FE
:10041000806480937A0080917A0084FFFCCF2091E1
:100420007800809179009927982F8827820F911D55
:10043000480F591F3F5F383048F38B98839880915D
:100440007A008F7780937A00CA0123E0959587958B
:100450002A95E1F7089580937C0083E880937A00E1
:100460000E94F30108959F92AF92BF92CF92DF92C4
:10047000EF92FF920F931F93CF93DF93C0E0D0E0F2
:1004800099240E94F3019C0180917C00882309F04B
:100490009DC080910001833009F04CC083E02B3275
:1004A00038078CF0AE01FA01EC50FE4F8591949123
:1004B0008217930730F493944E5F5F4F99E199153B
:1004C00090F76DE216C0E3E020323E078CF4AE01F7
:1004D000FA01EE5EFD4F859194912817390730F4AB
:1004E00093944E5F5F4FF3E6F91590F76BE201C00E
:1004F00060E281E00E947F06892D0E94F2039FE066
:10050000A92EA82220E3A20E182F12951F70120FF9
:1005100060E280E00E947F06612F82E00E947F06F9
:100520006A2D83E00E947F066AE284E00E947F06D3
:1005300063E447C0843009F049C1E92DFF27EE0F7D
:10054000FF1FE652FF4F859194918217930720F089
:1005500093948DE8891588F7892D0E940304EC0196
:1005600093E6991560F46BE280E00E947F068D2F80
:10057000992787FD9A95182F105D612F05C060E2BD
:1005800080E00E947F066BE281E00E947F060FE020
:10059000A02EAC22E0E3AE0E14E0D595C7951A95D7
:1005A000E1F78C2F8F708E0F682F82E00E947F06FC
:1005B0006A2D83E00E947F066AE284E00E947F0643
:1005C00066E485E00E947F0660E0FDC080917C00CB
:1005D000813009F0BFC0E90182E00E942B020E9435
:1005E000F3019C0140E050E0FA01E055FF4F859196
:1005F00094918217930730F493944E5F5F4FF6E126
:10060000F91590F7992029F486EF98E2A4E3B0E475
:1006100019C025E1291528F48AEB99E4ACE3B0E48C
:1006200011C0292D3327220F331F220F331F245AC5
:100630003F4FF901E590F490F9013296059114913C
:10064000D801C7018093010190930201A093030197
:10065000B0930401A1E09A2E90927C00CE01AA27CB
:1006600097FDA095BA2FBC01CD010E94A8127B0175
:100670008C018091010190910201A0910301B09140
:1006800004019C01AD01C801B7010E94FD12DC010B
:10069000CB0120E030E040E85AE3BC01CD010E94EC
:1006A000FD12DC01CB0120E030E040EC50E4BC0165
:1006B000CD010E94FD127B018C010E948B125B0117
:1006C0006C01862F9927AA2797FDA095BA2FBC0108
:1006D000CD010E94A812DC01CB019C01AD01C80133
:1006E000B7010E944812DC01CB0120E030E048EC69
:1006F00052E4BC01CD010E94FD12DC01CB01BC0122
:10070000CD010E948B127B018C018A2D0E94F20385
:10071000FFE0AF2EA822F0E3AF0E8E2D0E94F20371
:10072000182F12951F70105D60E280E00E947F0616
:1007300060E2892D0E947F0660E282E00E947F06CF
:100740006A2D83E00E947F0666E584E00E947F06B2
:10075000612F37CFC0917C00C230C1F58091790004
:100760000E94F20380917800982F9F70E0E3AE2EF4
:10077000A90E29E32A1518F477E3A72EA90E682FEE
:1007800062956F70162F105D1A3308F0195F61E4DF
:10079000892D0E947F0664E481E00E947F0663E465
:1007A0008C2F0E947F0680917900805D682F83E006
:1007B0000E947F06612F84E00E947F066A2D85E0FB
:1007C0000E947F06692D86E00E947F06DF91CF910F
:1007D0001F910F91FF90EF90DF90CF90BF90AF905F
:1007E0009F900895282F80E02A3018F08F5F2A50BC
:1007F000FBCF992734E0880F991F3A95E1F7282B12
:10080000822F9927089520E030E0843620F02F5F72
:100810003F4F8456FACF54E0220F331F5A95E1F729
:100820008A3020F02F5F3F4F8A50FACF44E0220FEA
:10083000331F4A95E1F79927822B932B0895209A2D
:10084000229A239A259A85B1806D85B91DB88EB1FB
:100850008C608EB98CE080936B0080ED80936C008F
:1008600080EC8CBB8DBB0E94E111809355010895F3
:1008700023B12095207D8CB180958C70282B822F00
:10088000992786FF02C094E00FC027FF02C095E0C1
:100890000BC082FF02C093E007C083FF02C092E05A
:1008A00003C084FF16C091E080914001882389F045
:1008B00080913E01882359F490933F0181E0809319
:1008C0003E0180914A01882311F00E942E1210925D
:1008D000400180EC8CBB10924C0108951F920F9246
:1008E0000FB60F9211242F933F934F935F936F9303
:1008F0007F938F939F93AF93BF93EF93FF930E9448
:100900003804FF91EF91BF91AF919F918F917F91AB
:100910006F915F914F913F912F910F900FBE0F906C
:100920001F9018951F920F920FB60F9211242F93BC
:100930003F934F935F936F937F938F939F93AF9367
:10094000BF93EF93FF930E943804FF91EF91BF9103
:10095000AF919F918F917F916F915F914F913F9157
:100960002F910F900FBE0F901F901895F8948091C3
:100970003E01882321F080913F0110923E0178943E
:1009800099270895F999FECFF89492BD81BDF89A00
:10099000789480B599270895F999FECFF89492BD7F
:1009A00081BD60BDFA9AF99AF999FECF78940895BD
:1009B00081118FEFE7E5F1E093E18193915097FF8B
:1009C000FCCF089580E00E94D8048FE08093E70078
:1009D00087EB8093E50087E08093E60080EC8093CE
:1009E000E4008091E40088608093E4001092460166
:1009F0000895E82F20E030E0663090F58A52813586
:100A000058F4E13608F0EF7DEA52FF27EE0FFF1FA2
:100A1000E457FD4F25913491862F992780FF02C01E
:100A20005FE001C050EF6695E62FFF27E95AFE4FC1
:100A3000BC016170707043E0922F9F7084E0369526
:100A400027958A95E1F76115710511F09295907FD0
:100A500080818523892B80833596415047FFECCFD9
:100A600008951F920F920FB60F921124DF92EF920A
:100A7000FF920F931F932F933F934F935F936F9327
:100A80007F938F939F93AF93BF93CF93EF93FF93F6
:100A9000DD2480914001882361F4809147018F5FBC
:100AA00080934701843028F081E080934001D09208
:100AB000470180914901833071F4809148018F5F33
:100AC00080934801813148F081E0809349018FE0B3
:100AD0008093480102C01092480180910501815025
:100AE0008093050190915601992371F0882371F448
:100AF00080914501882321F481E08093460106C05E
:100B000081508093450102C090938401FF2490910D
:100B10004601913009F06CC080914401853010F499
:100B2000EF2C01C0E92EC0E000E010E080918401CC
:100B3000992787FD9095800F911F97FD17C0FF2083
:100B4000A9F480918401992787FD9095F801E559D2
:100B5000FE4FE80FF91F8081DF2C87FF02C091E074
:100B6000D92E8F7721F4FC2EF39401C080E2DD2092
:100B700029F0EE2019F06C2F80E201C06C2F0E944A
:100B8000F904CF5F0F5F1F4FC63080F2ACEEB0E0CC
:100B9000E7E5F1E0C3E181918D93C150C7FFFBCF41
:100BA00080914301811181E08093F40080914201A2
:100BB0009091F900882311F0916001C09E7F90937D
:100BC000F900809141019091EE00882311F090622C
:100BD00001C09F7D9093EE0081E0F81611F48AEF3A
:100BE00003C0809184018F5F80938401109246013D
:100BF00080910501882319F483E080930501809199
:100C000044018A3019F41092440103C08F5F80932D
:100C10004401FF91EF91CF91BF91AF919F918F913F
:100C20007F916F915F914F913F912F911F910F9104
:100C3000FF90EF90DF900F900FBE0F901F901895D0
:100C4000FC01809146018823E1F7982F8491882345
:100C500091F0AF01ABE6B1E09F01F90184918D9372
:100C60009F5F2F5F3F4F4F5F5F4FFA018491882353
:100C700011F0993190F3E92FFF27E559FE4F1082CB
:100C8000973048F081E0809356011092840183E010
:100C90008093450104C0109256011092840181E0B6
:100CA000809346010895DC01E0914601EE23E1F7CF
:100CB0009E2F8C91882359F0FD01ABE6B1E0819124
:100CC0008D939F5F8081882311F09931C0F3E92FC4
:100CD000FF27E559FE4F1082973048F081E080935E
:100CE00056011092840183E08093450104C0109264
:100CF00056011092840181E0809346010895893164
:100D000028F4E82FFF27E559FE4F6083089590E20D
:100D1000EBE6F1E088E19193815087FFFCCF0895E5
:100D2000809343010895909146019923E1F76093E0
:100D300056019093840180934601089510924401D6
:100D4000089501972FEF8F3F920731F02CE70000B5
:100D5000215027FFFCCFF5CF0895CF93C0E080E866
:100D60008093610083E080936100C093700088E00D
:100D70008093B60088EC8093B300C0936E0081E04E
:100D8000809381008093B0008091B600282F332794
:100D9000217030708091B600992784709070282B54
:100DA000392B232B89F788EE93E00E94A1064FEFA1
:100DB00051E0F89446BB47BB109285001092840026
:100DC0001092B200B99BFECF109281007894B09B34
:100DD00003C02FEF3FEF0AC09091840080918500FF
:100DE000282F3327322F2227290F311D88E12B3658
:100DF000380724F080916600815006C0285E374194
:100E000034F4809166008F5F8093660001C0C1E07A
:100E100050938100CC2369F2CF9108950E94AD06D2
:100E200090E89093610083E08093610090BF87E039
:100E300080937F008FE085B980EF8EB9259A2D9A37
:100E40000E941F040E94220D0E9452118CE090E02B
:100E50000E940D120E94E2040895CFEFD4E0DEBF9D
:100E6000CDBF0E940E07789482E080937C000E94A0
:100E70002B020E94F30110928C0180E090E00E940E
:100E8000C204992790938601809385018F3F910535
:100E900021F4109286011092850181E090E00E9479
:100EA000C204992790939401809393018F3F9105F9
:100EB00021F4109294011092930182E090E00E943C
:100EC000C204992790938B0180938A018F3F9105EB
:100ED00021F410928B0110928A0183E090E00E942D
:100EE000C204992790938E0180938D018F3F9105C5
:100EF00021F410928E0110928D0184E090E00E9406
:100F0000C204992790938801809387018F3F9105B0
:100F100021F4109288011092870185E090E00E94F0
:100F2000C204809389018F3F11F41092890180914E
:100F3000890180934A0186E090E00E94C2049927CB
:100F40009093900180938F018F3F910521F410922F
:100F5000900110928F0187E090E00E94C20480937C
:100F600095018F3F11F4109295010E943F120E944B
:100F7000B604F82E80914C0190914D014E9720F0CF
:100F800088E180936000FFCF80918F019091900164
:100F9000009709F42B9A8130910509F42B98029758
:100FA00081F482E080937C000E942B020E94F30176
:100FB00023E0893E92070CF02B98885D93400CF457
:100FC0002B9A20918F01309190012330310579F4D3
:100FD000FF2021F030939701209396018091960194
:100FE00090919701892B11F02B9801C02B9A609159
:100FF0008C01662369F488EF92E00E94200654E099
:10100000F51609F4FBC485E0F81609F016C586C08C
:101010006A3099F460E08EEF92E00E94200624E0AE
:10102000F21609F4EBC445E0F41609F465C052E089
:10103000F51609F002C58BE0E7C4643191F460E075
:1010400083E093E00E94200684E0F81609F466C06D
:1010500025E0F21609F469C342E0F41609F0EDC484
:1010600051C06E3191F460E087E093E00E94200669
:1010700054E0F51609F440C085E0F81609F4BEC442
:1010800022E0F21609F0D9C44BC36832C1F460E023
:101090008BE093E00E94200644E0F41609F445C377
:1010A00055E0F516D9F182E0F81609F4B3C421E051
:1010B000F21609F0C2C488E180936000FFCF663168
:1010C00079F460E082E193E00E9420062A9A43E0EE
:1010D000F41691F051E0F51609F0AFC485E194C41F
:1010E000653191F460E088E193E00E9420062A983F
:1010F00083E0F81619F42A9A84E186C421E0F216F6
:1011000009F09BC486E180C46B30A1F560E08FE1FB
:1011100093E00E94200643E0F41611F48AE074C4C0
:1011200051E0F51609F089C48CE080938C01809120
:101130008701909188019093920180939101209171
:101140009301309194018CE390E0289FA001299FA6
:10115000500D389F500D112480918501909186018A
:10116000840F951F019690939A01809399010E9494
:10117000521163C46C3009F077C02A9881E00E9454
:10118000900610924D0110924C01209199013091DE
:101190009A012330310559F4309397012093960139
:1011A00080919501882319F081EC80938000223092
:1011B000310519F4109280002FC0232B69F580911E
:1011C00091019091920101979093920180939101E6
:1011D000892B41F42A9A8BE080938C0180E00E9455
:1011E00090061AC08DE080938C0120918D01309182
:1011F0008E018CE390E0289FA001299F500D389F1D
:10120000500D112480918A0190918B01840F951FBC
:1012100090939A01809399012091990130919A01BC
:10122000C9016CE370E00E944813FB01C9016CE343
:1012300070E00E9448138C018E2F0E94F203C82F89
:101240005FE0E52EE82250E3E50EC295CF70C50FB2
:10125000802F0E94F203082F182F1F70105D029537
:101260000F70005D63E559C06D3009F07DC02A9AAA
:1012700010924D0110924C018091990190919A0128
:10128000892BE9F48CE080938C01209193013091BB
:1012900094018CE390E0289FA001299F500D389F76
:1012A000500D11248091850190918601840F951F26
:1012B000019690939A01809399010E945211E091B6
:1012C0009901F0919A01E330F10521F4F09397012F
:1012D000E0939601CF016CE370E00E9448139B01FC
:1012E000CF016CE370E00E9448138C01822F0E94B2
:1012F000F203C82F4FE0E42EE82250E3E50EC2953A
:10130000CF70C50F802F0E94F203082F182F1F7077
:10131000105D02950F70005D67E580E00E947F061A
:1013200060E281E00E947F066C2F82E00E947F06CF
:101330006E2D83E00E947F06602F84E00E947F066E
:10134000612F85E00E947F0660E086E00E947F06B4
:1013500083E0F81609F071C32A9A8BE080938C0120
:1013600080E00E94900669C36F31B9F460E086E2C4
:1013700093E00E94200624E0F21609F4DFC045E065
:10138000F41609F4C8C153E0F51609F4CEC182E0A1
:10139000F81609F052C381E237C3613209F051C037
:1013A00081E00E94900681E08093410124E0F216E2
:1013B00031F48091850190918601019608C045E045
:1013C000F41649F4809185019091860101979093DC
:1013D0008601809385018091850190918601CC974B
:1013E00034F08BE390E090938601809385018091A7
:1013F00085019091860197FF04C01092860110929A
:1014000085018F2D8250823058F482E280938C01C6
:10141000109241016091850180E090E00E94CC042F
:1014200051E0F51609F062C08FE180938C0180E0F5
:101430000E949006109241016091850180E090E049
:1014400053C0623209F06CC081E00E94900681E0D6
:101450008093420124E0F21631F48091930190913F
:101460009401019608C045E0F41649F48091930177
:1014700090919401019790939401809393018091AE
:101480009301909194018436910534F083E690E0C5
:101490009093940180939301809193019091940192
:1014A00097FF04C010929401109293018F2D8250E7
:1014B000823058F481E280938C0110924201609155
:1014C000930181E090E00E94CC0451E0F51671F4A4
:1014D0008FE180938C0180E00E949006109242017F
:1014E0006091930181E090E00E94CC04809193018F
:1014F0000E94F203C82F3FE0E32EE82280E3E80ECB
:10150000C295CF70C80F809185010E94F203082F09
:10151000182F1F70105D02950F70005D63E587C086
:101520006032C1F460E08CE293E00E94200624E087
:10153000F21609F4F5C045E0F41611F485E264C230
:1015400053E0F51609F4F1C082E0F81609F075C20F
:1015500083E25AC2633209F07FC081E00E949006A4
:1015600081E08093410124E0F21631F480918A01F8
:1015700090918B01019608C045E0F41649F48091E2
:101580008A0190918B01019790938B0180938A013E
:1015900080918A0190918B01CC9734F08BE390E09D
:1015A00090938B0180938A0180918A0190918B01A5
:1015B00097FF04C010928B0110928A018F2D8250E8
:1015C000823058F484E280938C0110924101609142
:1015D0008A0182E090E00E94CC0451E0F51671F49B
:1015E00080E280938C0180E00E949006109241017D
:1015F00060918A0182E090E00E94CC0480918D018C
:101600000E94F203C82F2FE0E22EE82280E3E80ECA
:10161000C295CF70C80F80918A010E94F203082FF3
:10162000182F1F70105D02950F70005D67E580E058
:101630000E947F0660E281E00E947F066C2F82E0BC
:101640000E947F066E2D83E00E947F06602F84E05B
:101650000E947F06612FCEC0643209F052C081E043
:101660000E94900681E08093420124E0F21631F45A
:1016700080918D0190918E01019608C045E0F4168D
:1016800049F480918D0190918E01019790938E0184
:1016900080938D0180918D0190918E01843691050A
:1016A00034F083E690E090938E0180938D018091D9
:1016B0008D0190918E0197FF04C010928E011092BF
:1016C0008D018F2D8250823058F483E280938C01FB
:1016D0001092420160918D0183E090E00E94CC0461
:1016E00051E0F51609F08ACF80E280938C0180E00A
:1016F0000E9490061092420160918D0183E090E07B
:101700007BCF6532D1F460E081E393E00E94200654
:1017100024E0F21611F480E277C145E0F41611F4EA
:101720008FE172C153E0F51611F48EE16DC182E0D4
:10173000F81609F082C186E267C1663209F062C01C
:1017400024E0F21631F4809187019091880101968E
:1017500008C045E0F41649F4809187019091880112
:1017600001979093880180938701809187019091E0
:1017700088018436910534F083E690E090938801E7
:1017800080938701809187019091880197FF04C021
:10179000109288011092870151E0F51649F485E214
:1017A00080938C016091870184E090E00E94CC04DA
:1017B000809187010E94F203C82F9FE0E92EE82262
:1017C00080E3E80EC295CF70C80F63E480E00E940A
:1017D0007F0660E281E00E947F0660E282E00E9474
:1017E0007F0660E283E00E947F066C2F84E00E9407
:1017F0007F066E2D85E00E947F0660E086E00E94F5
:101800007F061BC16932B9F460E087E393E00E9470
:10181000200623E0F21609F4F1C042E0F41611F4B8
:101820008AE2F2C055E0F51609F486C084E0F816A5
:1018300009F003C17BC06A3221F5609195016623EE
:1018400021F060E08EE393E002C081E493E00E9427
:10185000200623E0F21649F489E280938C0160911E
:10186000950187E090E00E94CC044CEFF40E51E02B
:101870005F1508F4E2C0809195018527809395015A
:10188000DCC06B32B9F460E085E493E00E9420068E
:1018900083E0F81609F4B2C022E0F21611F48CE2EB
:1018A000B3C045E0F41609F4BAC054E0F51609F0E7
:1018B000C4C0B0C06C3239F560918901662321F053
:1018C00060E08BE493E002C08EE493E00E94200687
:1018D00083E0F81661F48BE280938C01809189019A
:1018E00080934A01682F85E090E00E94CC042CEFA1
:1018F000F20E41E04F1508F4A0C0809189018427C1
:10190000809389019AC06D32C9F460E082E593E06A
:101910000E94200653E0F51609F470C082E0F81624
:1019200011F48EE271C025E0F21611F48FE26CC062
:1019300044E0F41609F081C08BE266C06E3209F013
:1019400053C02115310521F460E086E593E014C011
:101950002130310521F460E08AE593E00DC02230AA
:10196000310521F460E08DE593E006C023303105B8
:1019700029F460E083E693E00E94200653E0F51628
:1019800051F48DE280938C0160918F0186E090E0AC
:101990000E94CC0452C085E0F81689F480918F0132
:1019A0009091900101969093900180938F010497FC
:1019B0000CF443C01092900110928F013EC024E0BD
:1019C000F216D9F580918F01909190010197909333
:1019D000900180938F0197FF30C083E090E0909357
:1019E000900180938F0129C06F32D9F460E088E6BE
:1019F00093E00E94200643E0F41611F488E204C04C
:101A000052E0F51621F480E380938C0116C085E046
:101A1000F81611F489E2F8CF24E0F21671F48DE2A1
:101A2000F3CF603351F443E0F41619F48FE280935E
:101A30008C0110927C000E94330260E081E00E94E1
:101A4000930695CA88EE93E00E94A106F8948091CF
:101A500070008E7F8093700088E08093B6001092B3
:101A6000B2008091B00085608093B0008091B60094
:101A7000282F3327217030708091B6009927847009
:101A80009070282B392B232B89F78FEF87BB809100
:101A90007000816080937000789410929A01109287
:101AA000990110929F018CE0809398018BE18093C3
:101AB0009B0188E080939E0184E090E090939D01DB
:101AC00080939C010895DF92EF92FF920F931F93F2
:101AD000CF9380911301882341F480919801E82FDE
:101AE000FF27EC5EFE4F808102C0809198010E942A
:101AF000F203C82F2FE0D22ED82280E3D80EC29551
:101B0000CF70C80F80919F010E94F203082F9FE0C1
:101B1000E92EE82280E3E80E02950F70080F80910D
:101B200099010E94F203182F8FE0F82EF12280E332
:101B3000F80E12951F70180F6C2F80E00E947F0620
:101B40006D2D81E00E947F06602F82E00E947F065B
:101B50006E2D83E00E947F06612F84E00E947F0645
:101B60006F2D85E00E947F0660E086E00E947F0680
:101B700081E00E94900660E081E00E94930680E090
:101B800090E0CF911F910F91FF90EF90DF9008951B
:101B9000CF92DF92EF92FF920F931F93CF93C82EB5
:101BA00080913901882361F08091980180934E01E2
:101BB00080919F0180934F01809199018093500102
:101BC00080911301882341F480914E01E82FFF2773
:101BD000EC5EFE4F808102C080914E010E94F203B4
:101BE000C82F5FE0F52EF82280E3F80EC295CF7083
:101BF000C80F80914F010E94F203182F4FE0E42E8E
:101C0000E82280E3E80E12951F70180F80915001B2
:101C10000E94F203082F3FE0D32ED82280E3D80E93
:101C200002950F70080F6C2F772780915101882340
:101C300009F4606880E00E947F066F2D772780910D
:101C40005101882309F4606881E00E947F06612FBA
:101C5000772780915101813009F4606882E00E9409
:101C60007F066E2D772780915101813009F46068DD
:101C700083E00E947F06602F772780915101823098
:101C800009F4606884E00E947F066D2D77278091BB
:101C90005101823009F4606885E00E947F0660E0AF
:101CA00086E00E947F0681E00E949006CC2011F021
:101CB0000E949E0660E081E00E94930681E080938E
:101CC000390184E0C81649F480915101E82FFF27BB
:101CD000E25BFE4F80818F5F0BC085E0C81651F438
:101CE00080915101E82FFF27E25BFE4F80818150F8
:101CF00080832CC083E0C81641F480915101882371
:101D000011F482E00AC0815008C082E0C81641F494
:101D1000809151018230C1F08F5F8093510116C0D4
:101D200081E0C81699F4F89480914E01809398014F
:101D300080914F0180939F0180915001992790934A
:101D40009A018093990178941092510180914E01EB
:101D50008F3F19F487E180934E0180914E018831C5
:101D600010F010924E0180914F018F3F19F48BE3D8
:101D700080934F0180914F018C3310F010924F01EE
:101D8000809150018F3F19F48BE380935001809133
:101D900050018C3310F0109250011092390180E004
:101DA00090E0CF911F910F91FF90EF90DF90CF9037
:101DB0000895CF93C82F80913A01882371F0109233
:101DC0003A0160911301613019F484E993E003C092
:101DD00061E088E993E00E942006C43081F46091BC
:101DE0001301613029F4109213018CE993E019C0BA
:101DF00081E080931301682F80EA93E012C0C53020
:101E000099F480911301882339F481E080931301C0
:101E1000682F84EA93E005C01092130161E088EA1C
:101E200093E00E94200604C0C13011F4C0933A012F
:101E300080E090E0CF910895AF92BF92CF92DF9271
:101E4000EF92FF920F931F9380919C010E94F203E7
:101E5000F82EEFE0CE2EC82280E3C80EF694F6945A
:101E6000F694F694F80E80919E010E94F203E82EFB
:101E70007FE0B72EB82280E3B80EE694E694E694AD
:101E8000E694E80E80919B010E94F203D82E6FE049
:101E9000A62EA82280E3A80ED694D694D694D694E3
:101EA000D80E80914B01E82FFF2707E011E0EE0FDD
:101EB000FF1FE00FF11F0190F081E02D84916F2D45
:101EC0000E947F0680914B01E82FFF27EE0FFF1F36
:101ED000E00FF11F0190F081E02D319684916C2D7F
:101EE0000E947F0680914B01E82FFF27EE0FFF1F16
:101EF000E00FF11F0190F081E02D329684916E2D5C
:101F00000E947F0680914B01E82FFF27EE0FFF1FF5
:101F1000E00FF11F0190F081E02D339684916B2D3D
:101F20000E947F0680914B01E82FFF27EE0FFF1FD5
:101F3000E00FF11F0190F081E02D349684916D2D1A
:101F40000E947F0680914B01E82FFF27EE0FFF1FB5
:101F5000E00FF11F0190F081E02D359684916A2DFC
:101F60000E947F0660E086E00E947F0681E00E947A
:101F7000900660E081E00E94930680E090E01F916F
:101F80000F91FF90EF90DF90CF90BF90AF900895AA
:101F9000FF920F931F93CF93F82E80913B018823DC
:101FA00061F080919C018093520180919E01809309
:101FB000530180919B0180935401C0913C01CC233B
:101FC000C9F4809152010E94F203182F082F0F705C
:101FD000005D12951F70105D60E28C2F0E947F06DD
:101FE00060E281E00E947F0669E582E00E947F0650
:101FF00069E535C0C130C9F4809153010E94F203F4
:10200000182F082F0F70005D12951F70105D60E291
:1020100080E00E947F0660E28C2F0E947F066DE4C4
:1020200082E00E947F066DE41AC0C23019F58091EB
:1020300054010E94F203182F082F0F70005D1295B3
:102040001F70105D60E280E00E947F0660E281E028
:102050000E947F0664E48C2F0E947F0664E483E084
:102060000E947F06612F84E00E947F06602F85E03A
:102070000E947F0660E086E00E947F0680E00E946A
:102080009006FF2011F00E949E0660E081E00E9411
:10209000930681E080933B0184E0F81649F4809137
:1020A0003C01E82FFF27EE5AFE4F80818F5F0BC067
:1020B00085E0F81651F480913C01E82FFF27EE5A95
:1020C000FE4F8081815080832CC083E0F81641F45C
:1020D00080913C01882311F482E00AC0815008C03D
:1020E00082E0F81641F480913C018230C1F08F5FAC
:1020F00080933C0116C081E0F81699F4F894809121
:102100005201992790939D0180939C0180915301E6
:1021100080939E018091540180939B01789410924A
:102120003C01809152018F3F19F483E68093520164
:1021300080915201843610F0109252018091530127
:10214000882319F48CE080935301809153018D30E2
:1021500018F081E08093530180919E018230C9F490
:1021600020919C0130919D01C90183709070892B51
:1021700081F4C90164E670E00E944813892B39F4A8
:10218000C90160E971E00E944813892B11F4EDE167
:1021900007C080915301E82FFF27E45DFE4FE081E7
:1021A00080915401882311F4E093540180915401EB
:1021B000E81718F481E08093540110923B0180E00D
:1021C00090E0CF911F910F91FF900895CF93C82F6A
:1021D00080913D01882379F010923D0180914B015F
:1021E000E82FFF27EE0FFF1FE35FFE4F61E08081C6
:1021F00091810E942006C43049F480914B018230C5
:1022000018F010924B010DC08F5F09C0C530B9F4B2
:1022100080914B01882311F482E001C081508093AA
:102220004B0180914B01E82FFF27EE0FFF1FE35F6B
:10223000FE4F61E0808191810E94200604C0C13080
:1022400011F4C0933D0180E090E0CF9108951F927A
:102250000F920FB60F9211248F939F938091990143
:1022600090919A01019790939A018093990180919E
:10227000960190919701009729F00197909397010B
:102280008093960180914C0190914D01019690931D
:102290004D0180934C019F918F910F900FBE0F9035
:1022A0001F90189583E0E4EAF1E0119211928150B9
:1022B00087FFFBCF9FEFE0EAF1E083E0919381504D
:1022C00087FFFCCF82E080936E0086E287BD8CE0C2
:1022D00084BD08951F920F920FB60F9211240F9391
:1022E0001F932F933F934F935F936F937F938F939E
:1022F0009F93AF93BF93CF93EF93FF93C3E004EA11
:1023000011E0D801ED91FD918D01309709F009950B
:10231000C150C7FFF6CFE0EAF1E0C3E080818F3F14
:1023200021F0882311F081508083C1503196C7FF7E
:10233000F5CFFF91EF91CF91BF91AF919F918F9189
:102340007F916F915F914F913F912F911F910F91CD
:102350000F900FBE0F901F901895AC0120E0E4EA9B
:10236000F1E0819191918417950761F02F5F2430FE
:10237000C0F320E0E4EAF1E080819181892B29F427
:102380005183408381E090E008952F5F329624309E
:1023900098F380E090E008959C0140E0E4EAF1E0E9
:1023A000808191818217930729F41182108281E044
:1023B00090E008954F5F3296443090F380E090E0D3
:1023C000089590E0E92FFF27E056FE4F80819F5F40
:1023D0008F3F21F41082892F99270895943090F32C
:1023E00080E090E00895F894E82FFF27E156FE4F33
:1023F000608378940895F894E82FFF27E156FE4F04
:102400008081789499270895F894E82FFF27E15662
:10241000FE4F8FEF8083789408959C01832F992736
:102420008093C5002093C40082E08093C00080E1C7
:102430008093C10086E08093C2000895982F809118
:10244000C00085FFFCCF9093C60008958091C00026
:102450008823E4F78091C60099270895CF93C9E0B7
:102460002D9A81E090E00E94A1062D9881E090E0F5
:102470000E94A106C150C7FFF3CFCF9108951092DB
:10248000800089E08093810080E180938800089536
:102490005058192E84D001D06AC0BA17620773074A
:1024A00084079507B1F188F40EF410940B2EBA2F1F
:1024B000A02D062E622F202D072E732F302D082ED3
:1024C000842F402D092E952F502DFF275523B9F02D
:1024D000591B49F0573E98F0469537952795A79593
:1024E000F0405395C9F776F0BA0F621F731F841F2F
:1024F00030F4879577956795B795F040939517FADF
:102500000F2E0895BF1BBB27BA0B620B730B840BF6
:10251000F6CFDEF670C097FB4ED09F3738F0FEE95D
:10252000F91B982F872F762F6B2F05C061C09695CA
:10253000879577956795F150D0F73EF49095809503
:10254000709561957F4F8F4F9F4F0895E89403C01A
:1025500097FB0EF4F3DFB62F672F782F892F9EE9B4
:10256000002405C09A95BB0F661F771F881F112492
:102570009923A1F08823B2F79F3F59F0BB0F48F48D
:1025800021F4002011F460FF04C06F5F7F4F8F4F74
:102590009F4F881F9795879597F9089529C0052E15
:1025A000092607FA440F551F5F3F79F0AA27A517A0
:1025B00008F051E04795880F991F9F3F31F0BB27E6
:1025C000B91708F091E0879508959F919F91112484
:1025D0005CC097FB880F991F9F3F31F0BB27B9174D
:1025E00008F091E0879508959F919F9111244DC027
:1025F00066277727882799270895D1DF01D0B7CF9D
:10260000992339F0552329F09F575F57950F13F4FD
:102610009AF1F1CF91589F3FE1F3629FA12D0F9264
:10262000BB27639FA00DB11DEE27729FA00DB11DAA
:10263000EE1FAF93AA27649FB00DE11D739FB00DED
:10264000E11DAA1F6627829FB00DE11DA61F552719
:10265000749FE00DA11D551F839FE00DA11D561F06
:10266000849FA00D511D852F7A2F6E2F1F900F90E4
:1026700088231AF4939539F408C0000C111CBB1F71
:10268000661F771F881F012808959FEF80EC08952B
:10269000AA1BBB1B51E107C0AA1FBB1FA617B70788
:1026A00010F0A61BB70B881F991F5A95A9F78095A4
:0826B0009095BC01CD010895D5
:1026B800039A993940030F790373036D038D0386D9
:1026C800037F03010C0102030405060708090A0B2E
:1026D8000C0102030405060708090A0B001F1C1F4A
:0E26E8001E1F1E1F1F1E1F1E1F0101010201CB
:00000001FF
